:100000000C94EB010C940A020C940A020C940A0260
:100010000C940A020C940A020C940A020C940A0230
:100020000C940A020C940A020C94601E0C94361F65
:100030000C9434190C940A020C940A020C940A02CF
:100040000C940A020C940A020C940A020C940A0200
:100050000C940A020C94BC190C940A020C940A0227
:100060000C940A020C940A020C940A020C940A02E0
:100070000C940A020C940A020C940A020C940A02D0
:100080000C940A020C940A020C940A020C940A02C0
:100090000C940A020C940A02D504D504010501054A
:1000A000690587059F069F0692052B063C063C06C0
:1000B000A71FCE1FC620CE1FC6201A203D20C62057
:1000C0009420A3203A003B0029001E001F002000BE
:1000D00021002200230024002500260027002D00F7
:1000E0002E002A0053004700000001513C003D0053
:1000F0002B0014001A000800150017001C0018003F
:100100000C00120013002F00300028005F00600078
:10011000610055003E003F00E000040016000700AB
:1001200009000A000B000D000E000F003300340020
:1001300000005C005D005E005600000040004100D1
:10014000E1001D001B000600190005001100100051
:10015000360037003800E500310059005A005B00D6
:100160005700000042004300E2003500000000009C
:1001700000002C0000000000000000000000000053
:10018000390062000000630000000000010001006F
:10019000005C0100010001000100010001000100FC
:1001A0000100010001000100010001000100010047
:1001B0000000010001000100010001000100010038
:1001C0000100010001000100010001000100010027
:1001D0000100010001000100010001000100010017
:1001E0000100010001000100010001000100010007
:1001F00001000100010001000000010001000100F8
:1002000001000000010001000100010001000100E7
:1002100001000100010001000100010001000100D6
:1002200001000100010001000100000001000100C7
:1002300001000100000000000000010000000000BB
:1002400000000000000000000100010000000100AB
:100250000000000014035A002D003100350030006A
:1002600020005000430042000000220362006C00A6
:1002700069006E0064006100730073006100730028
:10028000730069006E00310031003100000004038A
:10029000090409023B00020100A0FA090400000160
:1002A000030101000921110100012240000705811D
:1002B00003080001090401000103000000092111E5
:1002C00001000122B600070582032000011201008F
:1002D0000200000008EDFE6060010001020001055F
:1002E000010902A10185020901A1000509190129DD
:1002F00008150025019508750181020501093009DD
:10030000311581257F9502750881060938158125EB
:100310007F950175088106050C0A38021581257F35
:10032000950175088106C0C005010980A1018503FA
:1003300019012AB700150126B70095017510810033
:10034000C0050C0901A101850419012AA0021501AB
:1003500026A002950175108100C005010906A101C2
:100360008506050719E029E715002501950875019F
:1003700081020507190029EF1500250195F0750187
:10038000810205081901290595057501910295015C
:1003900075039101C005010906A101050719E029AE
:1003A000E715002501950875018102950175088101
:1003B000010507190029FF150026FF00950675089D
:1003C000810005081901290595057501910295011E
:1003D00075039101C00011241FBECFEFD0E2DEBF34
:1003E000CDBF11E0A0E0B1E0E8EFF2E400E00BBF28
:1003F00002C007900D92A439B107D9F722E0A4E911
:10040000B1E001C01D92A63FB207E1F70E94FB12C6
:100410000C947A210C94000081E0089581E0089505
:100420000C940E0208950C9412021F93CF93DF9345
:1004300000D000D01F92CDB7DEB749835A836B83BB
:100440003091970189819A81311114C0662359F046
:10045000222349F00E94DC08182F682F89819A8195
:100460000E94850803C00E94B008182F69817A8114
:10047000812F04C00E94DC0869817A810F900F905F
:100480000F900F900F90DF91CF911F910C9445101A
:10049000FC01262F408151816281738184810C94FB
:1004A000150281E00895CF93DF93EC0160E00E9494
:1004B0004802BE01DF91CF910C9413020C948E116F
:1004C0000C948A1108950E942F070E9462022FEF58
:1004D00084E39CE0215080409040E1F700C00000A0
:1004E0000C94E2190F931F93CF93DF938C0161E07B
:1004F0000E944802EC01B8010E9410028823F1F129
:10050000B801CE010E947D178823C1F1B801CE0148
:100510000E949115882391F1B801CE010E94D9164D
:10052000882361F1F8018281882309F1CB358DE5BB
:10053000D807C1F050F4C115FCE5DF0781F0CF3DCD
:10054000DC45A9F40E94130E19C0CC35EDE5DE0799
:1005500061F0CD35DD4559F40E94560D08C00E946A
:1005600063020CC00E945F0D02C00E94620DC801B0
:10057000DF91CF911F910F910C940C0280E0DF91DD
:10058000CF911F910F9108950E9414190C94F802B5
:100590000E94FB020C941A1908950C94CC0281E07D
:1005A0000895CF93C82F0E94CF02882379F0C0FF0F
:1005B00002C0779A01C07798C1FF02C0289A01C093
:1005C0002898C2FF02C0769A01C07698CF9108950C
:1005D0006F9A7798209A28986E9A76980895CF9374
:1005E000C82F0E94CD028C2F0E94D102CF91089576
:1005F00080E00C94EF020E94D9170C94EF020E9445
:10060000D91790919601891721F0809396010C9447
:10061000EF020895CF93DF93CDB7DEB72B970FB6D8
:10062000F894DEBF0FBECDBF4F83588769877A87A6
:100630008B8761110E94A20C9E012F5F3F4F86E0C5
:10064000F90111928A95E9F785E0FE013796D90103
:1006500001900D928A95E1F789819A814C815D81A3
:10066000452B31F09F3F31F491E08F3F19F403C0E7
:1006700091E001C090E090FF09C049815A816B81EF
:100680007C818D819E810E94C30B05C0C9010E949F
:1006900051028111F2CF2B960FB6F894DEBF0FBE38
:1006A000CDBFDF91CF910895FC01808191810E949F
:1006B0001E090895CF93882309F4A4C0C82F823857
:1006C000C1F40E94D91781FD9DC069E380910201A8
:1006D000909103010E94CF180E94C40C2FEF81EE6D
:1006E00094E0215080409040E1F700C0000069E3B1
:1006F00019C0833801F50E94D91780FD83C063E5D6
:1007000080910201909103010E94CF180E94C40CB5
:100710002FEF81EE94E0215080409040E1F700C03F
:10072000000063E580910201909103010E94DA18B4
:10073000CF910C94C40C8438C1F40E94D91782FD67
:1007400061C067E480910201909103010E94CF187B
:100750000E94C40C2FEF81EE94E021508040904025
:10076000E1F700C0000067E4DDCF8CEF8C0F813A29
:10077000D0F46C2F80910201909103010E944F18D8
:10078000882349F06C2F80910201909103010E940F
:10079000DA180E94C40C6C2F809102019091030121
:1007A0000E94CF18C5CF80E28C0F883048F4C77004
:1007B00081E001C0880FCA95EAF70E94850CB8CF86
:1007C000EBE5EC0FE33040F4F0E0E95BFE4F8081B5
:1007D00090E0CF910C940D18E8E5EC0FE73150F460
:1007E000F0E0EE0FFF1FE75EFE4F80819181CF9119
:1007F0000C942318CD3E30F08C2F0E948013CF91A3
:100800000C945214CF910895882309F464C082385F
:1008100079F40E94D91781FF5EC069E380910201DB
:10082000909103010E94CF180E94C40C69E310C08C
:100830008338B1F40E94D91780FF4DC063E58091E1
:100840000201909103010E94CF180E94C40C63E53D
:1008500080910201909103010E94DA180C94C40C5B
:10086000843879F40E94D91782FF35C067E48091FB
:100870000201909103010E94CF180E94C40C67E40A
:10088000E7CF9CEF980F913A10F4682FE1CF90E2F8
:10089000980F983050F4877091E001C0990F8A95B5
:1008A000EAF7892F0E948B0CD9CF9BE5980F9330E4
:1008B00020F480E090E00C940D1898E5980F9731A3
:1008C00020F480E090E00C9423188D3E20F00E94EC
:1008D000DB130C94521408951F93CF93DF93182FBA
:1008E000EB010E945A03209741F08FE99FE00197A6
:1008F000F1F700C000002197F6CF812FDF91CF9153
:100900001F910C940404893319F060E070E002C078
:1009100060E570E00C946C04882321F00E94850C43
:100920000C94C40C0895882321F00E948B0C0C9425
:10093000C40C0895CF92DF92EF92FF920F931F9312
:10094000CF93DF937C01D62FC72FFC011281058145
:1009500002950F700E947B0C8823B9F01123A9F037
:100960008C2F807F803421F080E28D0F883068F0FA
:100970008091BC0282FD09C082E00E94240D0E9489
:100980007B0C91E0D82ED92601C0D12CCC2EC2945C
:100990008FE0C8228C2D90E08C30910508F0CFC1FB
:1009A000FC01E45BFF4F0C940E218C2F807FCF70F5
:1009B000882311F0C295C07F112399F0CC2309F44C
:1009C000AAC180E28D0F883010F0D11104C08C2FA5
:1009D0000E94850C03C08C2F0E94950C0E94C40CB1
:1009E0009AC18D2F0E940404CC2309F4A8C180E28F
:1009F0008D0F883038F1DD2329F18C2F0E949B0C5C
:100A000024C08C2F807FCF70803211F0C295C07FC0
:100A1000DD2319F0D130A1F13DC08091BC0282FFED
:100A200017C0112349F0CC2329F08C2F0E94850C8C
:100A30000E94C40C80E070C180E00E940404CC23BA
:100A400009F47DC18C2F0E948B0C0E94C40C77C1CD
:100A5000112371F0002341F0013031F40E94A50C04
:100A60008C2B0E94AD0C6BC10E94A50C8C2B1DC061
:100A7000002319F0013009F462C10E94BA0C25C0AC
:100A8000112321F0063008F05AC10EC0053008F0DD
:100A900056C11BC0112361F0002331F0F70185819D
:100AA00080FF39C18F7085838C2F0E948C0447C1D1
:100AB000002359F0D93309F03FC1FFEF07EE13E0EF
:100AC000F15000401040E1F735C18C2F0E94930493
:100AD00036C18C2F86958695837019F0813061F030
:100AE0002EC1112321F08D2F9C2F937002C080E026
:100AF00090E00E940D182BC1112321F08D2F9C2F07
:100B0000937002C080E090E00E94231820C18D2FD6
:100B1000112319F00E94801302C00E94DB130E946F
:100B2000521415C18C2F837009F047C011110BC1ED
:100B30002D2F229526952770220F220F6D2F6F7073
:100B4000862F90E0A0E0B0E0022E04C0880F991F2D
:100B5000AA1FBB1F0A94D2F7D4FF10C04FE050E089
:100B600060E070E004C0440F551F661F771F2A9590
:100B7000D2F7409550956095709503C040E050E0E5
:100B8000BA01C695C695C3708A019B01082B192B23
:100B90002A2B3B2BC901B801C23049F058F4C130AF
:100BA00019F00E949B07CFC00E948907CCC00E9409
:100BB000AD07C9C00E948707C6C0112319F08C2F4A
:100BC000817001C08695882309F4BDC02D2F229520
:100BD00026952770220F220F6D2F6F70862F90E0C1
:100BE000A0E0B0E0022E04C0880F991FAA1FBB1F0F
:100BF0000A94D2F7D4FF10C04FE050E060E070E0FC
:100C000004C0440F551F661F771F2A95D2F74095E1
:100C100050956095709503C040E050E0BA01C695CC
:100C2000C695C3708A019B01082B192B2A2B3B2BDD
:100C3000C901B801C23049F058F4C13019F00E941E
:100C4000600881C00E944E087EC00E9472087BC06E
:100C50000E94C10778C0CF70112339F08C2F0E94F9
:100C6000E7078D2F0E948C046EC08D2F0E94930485
:100C70008C2F0E94080867C0D23F21F128F4D03F92
:100C800041F0D13FC1F043C0D33F19F1D43F79F0D7
:100C90003EC0112341F0053008F051C08C2F8F71F8
:100CA0000E942D084CC0063008F049C0F7CF809153
:100CB000BC0282FF18C0112339F08C2F8F710E9463
:100CC000E7073DC01123C9F38C2F8F710E940808DC
:100CD00036C0112329F08C2F8F710E94D2072FC0AC
:100CE0000E94CD072CC0112349F0CF718C2F0E9498
:100CF000E70763E08C2F0E94090D21C081E00E946C
:100D0000240D0230E0F082E00E94240D18C011236F
:100D100031F0002391F28D2F0E945A0310C000235E
:100D200099F2D93349F41FEF27EE33E011502040F8
:100D30003040E1F700C000008D2F0E94040488EFCE
:100D40008C0D843020F40E94D9170E94EF02DD2020
:100D5000C9F00E94770C80FD15C0F70112820E9435
:100D6000710C0E94E707C7010E94E3060E94710C04
:100D7000DF91CF911F910F91FF90EF90DF90CF9077
:100D80000C940808DF91CF911F910F91FF90EF9085
:100D9000DF90CF9008950F931F93CF93DF93EC01D3
:100DA000688179818A810E9429098C010E948408C6
:100DB0000E947507B801CE010E949A04DF91CF917D
:100DC0001F910F910895CF93DF93EC019881898152
:100DD0002B813C81232B31F08F3F31F481E09F3F09
:100DE00019F403C081E001C080E080FD1DC0CE0188
:100DF0000E947202811110C00E947B0C8823A1F016
:100E00008A81882389F08091BC0282FD0DC082E036
:100E1000DF91CF910C94240DCE010E94CB06CE0120
:100E2000DF91CF910C945302DF91CF91089580E030
:100E300090E00E940D1880E090E00E9423180E942C
:100E4000A20C0E94C40C0E9483150C945214809131
:100E50000201909103010E94E5180C9417070E946B
:100E6000920C0C94270792959F70963079F010F4AD
:100E7000925001C09A50923068F4803F69F018F4A3
:100E8000883E40F409C0843F29F406C0883E20F023
:100E9000813F11F080E0089581E00895FC01808198
:100EA00091810E941E090E9433070895CF93DF931A
:100EB00000D000D01F92CDB7DEB70F900F900F90EB
:100EC0000F900F90DF91CF910895CF93DF9300D0D3
:100ED00000D000D0CDB7DEB726960FB6F894DEBFAF
:100EE0000FBECDBFDF91CF910895089508950C9462
:100EF00076070C9477070E9479076093DD01709361
:100F0000DE018093DF019093E0010C9417070C94AD
:100F10007B070F931F930091DD011091DE0120915B
:100F2000DF013091E001602B712B822B932B1F91FD
:100F30000F910C947B070F931F930091DD0110918B
:100F4000DE012091DF013091E001602371238223D3
:100F500093231F910F910C947B070F931F93009184
:100F6000DD011091DE012091DF013091E001602769
:100F70007127822793271F910F910C947B070C9464
:100F800076070E94BF076093D9017093DA018093BE
:100F9000DB019093DC010C94170760E070E0CB015B
:100FA0000C94C1070F931F9341E050E060E070E0A4
:100FB0008A019B0104C0000F111F221F331F8A9555
:100FC000D2F7C901B8011F910F910C94C1070F937B
:100FD0001F9341E050E060E070E004C0440F551FF3
:100FE000661F771F8A95D2F78091D9019091DA0117
:100FF000A091DB01B091DC018A019B01082B192B28
:101000002A2B3B2BC901B8011F910F910C94C107EA
:101010000F931F9341E050E060E070E004C0440F84
:10102000551F661F771F8A95D2F74095509560959A
:1010300070958091D9019091DA01A091DB01B09176
:10104000DC018A019B01082319232A233B23C901C0
:10105000B8011F910F910C94C1070F931F9341E0AA
:1010600050E060E070E004C0440F551F661F771F1A
:101070008A95D2F78091D9019091DA01A091DB0194
:10108000B091DC018A019B01082719272A273B27F9
:10109000C901B8011F910F910C94C1070F931F93C1
:1010A0000091D9011091DA012091DB013091DC012E
:1010B000602B712B822B932B1F910F910C94C107E6
:1010C0000F931F930091D9011091DA012091DB0158
:1010D0003091DC0160237123822393231F910F91B0
:1010E0000C94C1070F931F930091D9011091DA015D
:1010F0002091DB013091DC01602771278227932743
:101100001F910F910C94C107089524E1929F800DC7
:101110001124E82FE695E695E695877051E001C029
:10112000550F8A95EAF785E0E89FF0011124E8560B
:10113000FE4F20E030E070E04081CB01022E02C083
:10114000969587950A94E2F7817081958427852387
:10115000842781932F5F3F4F2530310569F708952C
:1011600024E1929F800D1124682F669566956695FF
:10117000982F977085E0689FB001112440E050E0FF
:1011800080E0FB01E40FF51FE856FE4F208130E0C0
:10119000092E02C0369527950A94E2F7217033276D
:1011A000042E01C0220F0A94EAF7822B4F5F5F4F93
:1011B0004530510531F70895BF92CF92DF92EF92FB
:1011C000FF920F931F93CF93DF938C01C090D901AF
:1011D000D090DA01E090DB01F090DC018091DD013C
:1011E0009091DE01A091DF01B091E001C82AD92AD7
:1011F000EA2AFB2ACFE1D0E0D701C6010C2E04C0B9
:10120000B695A795979587950A94D2F780FD04C067
:10121000219790F7B12C07C0BC2EB8018C2F0E94EB
:1012200058100197A9F38B2DDF91CF911F910F914A
:10123000FF90EF90DF90CF90BF900895CF93DF9312
:10124000EC010E94DC08BE010E945810DF91CF9192
:1012500008951F93CF93DF93EB019091970199230A
:1012600021F0CB010E941E0913C0882349F0CB0155
:101270000E94DC08182F682FCE010E94850804C048
:10128000CB010E94B008182FBE01812F0E94581078
:10129000DF91CF911F9108951F93CF93DF93C0915A
:1012A000E10116E08091E201C81799F0D0E01C9F9F
:1012B000F0011D9FF00D1124ED51FE4F4081518131
:1012C00062817381848195810E9465072196C77030
:1012D000E9CFDF91CF911F91089540911302509172
:1012E000140260911502709116028091170290917C
:1012F00018020C946507EF92FF920F931F93CF9300
:10130000DF938091180282958F7009F065C08091FB
:101310001502882309F460C08091E101F090E20198
:10132000109113020091140260911602709117023D
:1013300091E01F3F09F090E0C0910001D0910101C0
:10134000292F96E0E92E8F1509F446C06115710525
:1013500021F00F3F21F030E003C031E001C0322F17
:1013600090E030FD36C0E89EF001E99EF00D1124BA
:10137000DF01AD51BE4F11963C911197301329C03A
:101380003C91311326C012963C911297311121C025
:1013900013964D915C911497461B570B4C175D07A4
:1013A000C0F4809118028F70806180931802E85118
:1013B000FE4F80818F708061808383E192E00E9484
:1013C000E306DF91CF911F910F91FF90EF900C9466
:1013D0004C0901968770B7CFDF91CF911F910F9184
:1013E000FF90EF9008959F92AF92BF92CF92DF92BD
:1013F000EF92FF920F931F93CF93DF93CDB7DEB79A
:1014000061970FB6F894DEBF0FBECDBF8C0185E0AB
:10141000F801DE011D9601900D928A95E1F7D80141
:101420001296EC9090911302E09114022091160212
:10143000309117022115310531F0EF3F31F481E091
:101440009F3F19F403C081E001C080E0B82FB17064
:101450009B2E80FD47C1D8014C9111965C9111974C
:101460001396AD90BC90149783E1C82E82E0D82EDD
:10147000F0901502B501621B730B209100013091B1
:101480000101FF2009F4D9C0809118026217730787
:1014900008F095C0282F207F09F052C05E1313C0BA
:1014A000491311C0FE2CE1100EC08F708061809333
:1014B00018020E946D09C6010E94E306809118027D
:1014C000F80185834DC1AB2831F05F3F31F481E0F5
:1014D0004F3F19F403C081E001C080E080FD03C0EC
:1014E00081E08E2502C080E090E0F82FF170FF2EA1
:1014F00080FF1CC08091E1012091E20136E082175B
:1015000009F40BC190E0389FF001399FF00D1124D0
:10151000ED51FE4F6181561306C06081461303C032
:101520006281E61203C001968770E9CFFE2CEE209F
:1015300009F416C18091180281608093180254C08A
:101540005E1306C0491304C0E11002C0F80199C03F
:10155000C8010E944E07882361F1EE2051F12091CD
:101560001802822F82958F7090E0029774F080911C
:1015700013029091140298878F831986BB86AA86DE
:101580002C87CE0107960E94E30686E0F801A3E1CE
:10159000B2E001900D928A95E1F70E947B090E94CA
:1015A0006D090AC05E1711F1C8010E944E07811132
:1015B0002CC0C8010E94E306FF24F394D1C0282F59
:1015C000207F81F77A2DB98AA88A6E2D89890E9499
:1015D000560783E192E00E94E30686E0D6011D9261
:1015E0008A95E9F70E946D09F12CBAC04913DCCF46
:1015F000E110DACFF8018583C8010E94E30686E096
:10160000D6011D928A95E9F7ABC0EE2091F22091A8
:101610001802822F82958F7090E002970CF4B5CF5C
:1016200080911302909114029A8389831B82BD8258
:10163000AC822E83CE010196A6CF6217730708F005
:1016400044C0FE2CEE2009F4B4CF5E1330C0491321
:101650002EC02091180220FD21C0822F82958F700C
:10166000482F50E041155105C9F0F80125834F304E
:10167000510541F08F5F982F9295907F822F8F7048
:10168000892B8583C8010E94E30686E0F801A3E167
:10169000B2E001900D928A95E1F73CC086E0F80136
:1016A000A3E1B2E001900D928A95E1F759C0C8011B
:1016B0000E944E07811169CF80911802816080934A
:1016C0001802C8010E94E3064BC07A2DB98AA88A85
:1016D0006E2D89890E94560786E0D6011D928A9553
:1016E000E9F718C0EE2009F464CFC8010E944E0744
:1016F000F82E882309F45DCF86E0F801A3E1B2E07B
:1017000001900D928A95E1F783E192E00E945403E3
:101710000E947B090E946D0923C04D875E878D85DD
:101720009E850E941E09292F22952F70223028F4B1
:101730009F7039F0811105C00BC0243028F49F70D0
:1017400049F4805E883020F0C8010E94E3069F2C97
:10175000F92C06C0D80115969C91907F91F7F8CF8F
:101760008F2D61960FB6F894DEBF0FBECDBFDF910F
:10177000CF911F910F91FF90EF90DF90CF90BF908E
:10178000AF909F9008951F93CF93DF93CDB7DEB7AF
:101790002C970FB6F894DEBF0FBECDBF4F8358878E
:1017A00069877A878B879C87CE0107960E94F30909
:1017B0008823D1F09F8188852A853B85232B31F0B2
:1017C0008F3F31F481E09F3F19F403C081E001C0F5
:1017D00080E080FD47C04F81588569857A858B857B
:1017E0009C850E9465073EC086E0FE013796DE01BB
:1017F000119601900D928A95E1F7FF81E8856A853F
:101800007B856115710531F0EF3F31F481E0FF3FD9
:1018100019F403C081E001C080E080FD23C0209165
:10182000E20130E0C9010196877099274091E101FA
:1018300050E084179507F1F1F983EA837D836C8387
:1018400096E0929FD001939FB00D1124AD51BE4FF1
:10185000FE01319601900D929A95E1F78093E20195
:101860000E944C0916E08091E1019091E2018917F4
:1018700071F1189FC00111248D519E4F0E94F309F0
:10188000882329F1E091E1011E9FF0011124ED511F
:10189000FE4F4081518162817381848195810E94D4
:1018A00065078091E10190E0019687709927809308
:1018B000E101D9CF0E942F071092E2011092E101BD
:1018C000E3E1F2E086E0DF011D928A95E9F72C96CC
:1018D0000FB6F894DEBF0FBECDBFDF91CF911F9141
:1018E0000895809139028595859585950895809113
:1018F00039028770089590913902977081E009F458
:1019000080E0089580915C02089590915C02892B9B
:1019100080935C020895809590915C028923809366
:101920005C02089510925C02089590915B02892BED
:1019300080935B020895809590915B028923809348
:101940005B02089510925B02089580913A02089517
:1019500008950C94A80C0C94A90C9091BC0292FDD3
:1019600008C090913A02981721F080933A020C94A3
:10197000AB0C089580913A02882329F010923A0224
:1019800080E00C94AB0C0895CF93DF93E0910201BB
:10199000F091030180915C028083E0910201F0915B
:1019A0000301908180915B02892B808380913A02B0
:1019B000882381F0E0910201F09103019081892B4D
:1019C000808380910201909103010E943918811156
:1019D0000E94BA0CC0910201D091030140E250E094
:1019E00069E172E0CE010E942B21892B69F080E22F
:1019F000FE01A9E1B2E001900D928A95E1F7CE01D6
:101A0000DF91CF910C94E517DF91CF9108950C945D
:101A1000A80C9091BC0292FD10C098E0899F9001A3
:101A20001124262B209339020E94E7078091390266
:101A30008595859585950C94070D0C94E707109274
:101A4000390280E00C94070D2091390280958223A1
:101A500080933902982F977099F430E0482F082E20
:101A6000000C550B2417350759F09091BC0292FDDC
:101A700007C08595859585950E9408080C941F0DD3
:101A800008959091BC0292FB222720F9281769F053
:101A900080FB92F99093BC028091BB029091BC02B2
:101AA0000E948F0D82E00C94240D08958091BC0259
:101AB00082FB882780F991E089270C94410D81E011
:101AC0000C94410D80E00C94410D6FEF7FEF80E0AE
:101AD00090E00C94642180E090E00E94402121E09D
:101AE000893E9E4F09F020E0822F089582E090E029
:101AF0000C94382183E090E00C943821CF9384E05B
:101B000090E00E943821C82F82E290E00E943821A4
:101B10002C2F30E0A901582BCA01CF910895CF9303
:101B2000C92F682F84E090E00E9446216C2F82E24A
:101B300090E0CF910C944621AB01BC018FE090E086
:101B40000C945821AB01BC0183E190E00C94582126
:101B500060E070E0CB010C94A20D60E070E0CB017E
:101B60000E949C0D0C94A80D69EE7EEF80E090E041
:101B70000E94642160E082E090E00E94462160E0E3
:101B800083E090E00E9446211092DD011092DE0178
:101B90001092DF011092E00160E084E090E00E948A
:101BA000462160E082E290E00E94462160E085E00C
:101BB00090E00E94462160E086E090E00E9446218D
:101BC0006FEF87E090E00E94462140E050E0BA01CC
:101BD00088E090E00E94582160E08DE090E00E9453
:101BE000462140E050E0BA0188E190E00E9458218F
:101BF00060E087E190E00E94462140E050E0BA01B9
:101C00008CE190E00E94582160E070E080E290E07A
:101C10000E94642140E050E0BA0188E190E00E9417
:101C200058210C94AD0D0C94B40D682F8EE090E00B
:101C30000C9446210E94A11960937502709376025C
:101C4000809377029093780260937102709372028E
:101C50008093730290937402089585B7806885BF5E
:101C600085B7806885BF089581E008950C94340E8F
:101C700008950C94380E0C94380E0C943B0E0C9472
:101C8000380E0C943F0E0C94380E0E942D0E84E3F7
:101C900091E10E94CF170E94430E0C94410E0E94C6
:101CA000390E0C94380E0E944E110C94E8020E94DA
:101CB0008C190E9452120E94530EEBEBF2E08081CD
:101CC000806880838091BB029091BC020E948F0D3E
:101CD0000C943D0E2F923F924F925F926F927F92A3
:101CE0008F929F92AF92BF92CF92DF92EF92FF922C
:101CF0000F931F93CF93DF93CDB7DEB72D970FB61A
:101D0000F894DEBF0FBECDBF0E946712282E81114E
:101D10000E941A0E8DE592E09D878C8700E010E00E
:101D2000302E802F0E9472112B013C01EC85FD8525
:101D300081919191A191B191FD87EC87530142016D
:101D400088269926AA26BB2681149104A104B104F1
:101D5000B1F40F5F1F4F0530110511F78FEF898325
:101D60008A831B820E9495198160782F9D838C83C2
:101D700049815A816B818D810E940A0351C08091F3
:101D8000790281FD0E947E111B86C12CD12C760127
:101D9000C394D501C4018C219D21AE21BF21892B83
:101DA0008A2B8B2B91F10E94360E8823D1F0FB8574
:101DB000FE833F824C205D206E207F2081E04528FD
:101DC0004628472809F480E088870E949519816099
:101DD000782F9A8789874E815F8168858A850E94DE
:101DE0000A03000F111F000F111FF801E35AFD4FE6
:101DF00080819181A281B381C826D926EA26FB265B
:101E0000C082D182E282F3820BC08B858F5F8B8789
:101E1000CC0CDD1CEE1CFF1C843109F0BACF99CF2D
:101E200081E0211001C080E02D960FB6F894DEBF4E
:101E30000FBECDBFDF91CF911F910F91FF90EF901B
:101E4000DF90CF90BF90AF909F908F907F906F90DA
:101E50005F904F903F902F9008950E946A0E0E94CD
:101E600070140C94FF02CF93DF930E945D10EC017D
:101E7000811521E5920708F045C0811530E59307EB
:101E800008F094C0883E910528F5803E910508F041
:101E9000F8C0883A910570F4853A910508F07CC045
:101EA0008130910509F475C008F4E8C0049708F082
:101EB000E8C0E4C08F3B910508F0E0C0C85AD0E00C
:101EC000CC0FDD1FC65BDE4F0990D881C02DCE013F
:101ED0009464D8C0811540E2940758F4811551E00C
:101EE000950708F0CEC08D3E910508F4C7C09065F7
:101EF000C9C0C11580E4D80708F4C0C0DF70CE01A6
:101F0000906AC0C0811525E59207A8F4811534E5D3
:101F1000930708F095C0811543E5940708F07BC04E
:101F2000811552E5950708F061C0D82FCC27CE0166
:101F3000816F906AA7C0C11589E5D807A0F4C115C3
:101F400028E5D20708F082C0C11536E5D30708F0AE
:101F500095C08C2F0E94F1108F7190E0D82FCC2764
:101F6000CE0190628FC0C1154AE5D40708F474C051
:101F7000CE0190568115904208F080C08D2F8F7150
:101F80000E94F110DD27D0628F71AE01582BCA017B
:101F900079C081E090E076C0C55AD0E0C858DE4FE5
:101FA0008881C82FD0E0CE0190646CC074E0969513
:101FB00087957A95E1F7282F23703C2F337081E0C5
:101FC00090E002C0880F991F3A95E2F79C68AC0137
:101FD000522B9A019C2F9F709695969550E2959F53
:101FE000E0011124C9018C2B9D2B4CC083709927D3
:101FF00021E030E002C0220F331F8A95E2F79C2FC8
:102000009695969580E2989FE0011124C22BD32BE0
:10201000CE019C6837C08370992721E030E002C070
:10202000220F331F8A95E2F79C2F9695969540E2F2
:10203000949FE0011124C22BD32BCE019A6822C0B9
:10204000D82FCC27CE01846F906A1CC0DC2FCC2700
:10205000CE01806F906A16C08C2F8F700E94F11095
:1020600094E0D695C7959A95E1F7CF70D0E0DC2F34
:10207000CC27D0699E01282BC90104C080E090E0E4
:1020800001C0CE01DF91CF91089524E6829FC00167
:102090001124FC0124E1729FE00DF11D1124E60FD3
:1020A000F11DEE0FFF1FEC53FF4F859194910895A2
:1020B0000E9445100E94330F08958238910569F1FE
:1020C000B0F48133910509F46DC048F4893291056B
:1020D00009F463C08A32910509F469C00895853313
:1020E000910509F455C089339105B9F00895833EEF
:1020F000910569F138F4803E9105B1F0823E910579
:1021000009F10895863E9105A9F1873E9105B9F13F
:10211000843E910509F064C023C02091BB0220FDDC
:102120004FC021FD4DC008958091BB0280FD44C089
:102130008091BC0280FF44C08091BB0284FD42C0FC
:1021400083EE4DC08091BB0282FF38C0F5CF8091F5
:10215000BB0282FD33C08091BC0280FD31C0ECCF58
:102160008091BC0281FF32C08091BB0284FD2AC0F5
:1021700087EE35C08091BB0283FF26C0F5CF8091EA
:10218000BB0283FD21C08091BC0281FD1FC0ECCF4A
:102190008091BB0285FD1CC01DC08091BB0285FDE6
:1021A00019C016C08091BB0286FD16C017C0809171
:1021B000BB0286FD13C010C089E311C082EE0FC0C0
:1021C00080EE0DC080E00BC086EE09C084EE07C033
:1021D00089E205C085E303C08AE201C081E390E0A3
:1021E00008959091BB0292FF0DC0282F28712830CE
:1021F00019F4877F846006C0282F2471243011F4DD
:102200008B7F886093FF0DC0282F2871283119F427
:10221000877E846106C0282F2471243111F48B7EBF
:1022200088612091BC0220FF0DC0382F38713830F2
:1022300019F4877F816006C0382F3171313011F475
:102240008E7F886021FF0DC0282F2871283119F456
:10225000877E816106C0282F2171213111F48E7E85
:10226000886194FD877E089580E008950C94650D43
:102270000E9467128FE39CE90197F1F700C000000C
:102280000E94671280E00E94721160FF04C00E94E9
:1022900036110C94E21908950C9438110E946B0DBC
:1022A000811102C00E94130E0E94760D8093790264
:1022B0000E947E0D9093BC028093BB020E944C1141
:1022C0000E947A0D682F70E080E090E00E948707FE
:1022D0006091D9017091DA018091DB019091DC016C
:1022E0000C94BF0724E0829FC0011124FC01EF522F
:1022F000FD4F60817181828193810895089580EA04
:102300008A95F1F7089500C008950C947F110895FF
:102310000C9487110C9488110C9487110C948C11D7
:10232000F894E82FE295EF70F0E031A1282F2F709C
:1023300081E090E001C0880F2A95EAF7982F9095E8
:10234000932391A392A1892B82A3789408950F934C
:102350001F93CF93DF93CFE8D1E089918F3F11F0A6
:102360000E94901181E0C439D807B9F7CBE7D1E0DA
:102370000FE811E089918F3F11F00E9490110C1726
:102380001D07C1F7DF91CF911F910F9108954F92D3
:102390005F926F927F928F929F92AF92BF92DF92E5
:1023A000EF92FF920F931F93CF93DF938C01C62F71
:1023B000D0E0CE0181579E4F7C01FC0190819F3F70
:1023C00009F460C0D62EF894E92FE295EF70F0E0A2
:1023D00081A19F7021E030E001C0220F9A95EAF7B9
:1023E000822B81A382A12095282322A378940E9486
:1023F0008311EBE7F1E02FE831E0412C512C320161
:102400004394812C912C540181918F3F99F0A82FF6
:10241000A295AF70B0E090964C9150E08F70BA01E9
:1024200002C0759567958A95E2F760FD03C0D301F8
:10243000C20103C080E090E0DC01882A992AAA2A20
:10244000BB2A440C551C661C771C2E173F07E1F66F
:10245000F70180818F3F11F00E94901161E081149B
:102460009104A104B10409F460E08D2D0E9485114E
:10247000CC0FDD1FCC0FDD1FC00FD11F88829982CA
:10248000AA82BB82DF91CF911F910F91FF90EF90B5
:10249000DF90BF90AF909F908F907F906F905F90F4
:1024A0004F9008950E94A71184E1E1EDF2E0DF0171
:1024B000982F1D929A95E9F7EDEBF2E0DF011D925E
:1024C0008A95E9F785E00E94B2120C945E02FF92B1
:1024D0000F931F93CF93DF93CDB7DEB764970FB6FB
:1024E000F894DEBF0FBECDBF8E010F5F1F4F84E19A
:1024F000F80111928A95E9F7F12C6F2DC8010E941D
:10250000C711F394F5E0FF12F8CF44E150E0B801B1
:102510008DEB92E00E942B21FF24F394009709F4A5
:10252000F12C892B41F084E1F801ADEBB2E0019090
:102530000D928A95E1F72F2D45E061ED72E08DEB6C
:1025400092E00E94B3120E9460028F2D64960FB633
:10255000F894DEBF0FBECDBFDF91CF911F910F91D9
:10256000FF9008950895FF920F931F93CF93DF93E9
:10257000F82ED92F8B01C42F222349F081E08093BC
:102580007C020E94951990937B0280937A0280913D
:102590007C028823F1F080917A0290917B020E9464
:1025A000AD190597B0F0EF2DFD2FD80180E090E038
:1025B0004C2F50E08417950754F40191119121910B
:1025C00031910D931D932D933D930196F3CF10926E
:1025D0007C02DF91CF911F910F91FF9008950E948F
:1025E000B91B0E94570E0C94C51B0E94C91B0E9468
:1025F0002D0F0C94E31B0E9433190E94A01B0E9414
:10260000450E0E94EF120E94F5120E944F0EFBCF62
:102610008091830280FF06C06091090170E0660F1F
:10262000771F26C081FF04C06091090184E005C0C6
:1026300082FF07C06091090188E0689FB001112402
:1026400017C0909182029923D1F0609108019617EA
:1026500088F72091090188E0289F90011124929F1A
:10266000A001939F500D112470E0CA010E94FA202E
:102670006038710540F46115710519F406C068E011
:1026800070E0862F08958FE7089581E00895809186
:10269000830280FF08C06091050170E07595679521
:1026A0007595679521C081FF06C06091050170E0B6
:1026B0007595679519C082FF04C06091050170E0AF
:1026C00010C090918102992399F0609104019617AE
:1026D000A0F780910501899FC001112470E00E943C
:1026E000FA206038710540F46115710519F406C0CF
:1026F00061E070E0862F08958FE7089581E00895E6
:102700008D3E21F40E940813819504C08E3E29F469
:102710000E9408138093870208958F3E21F40E943F
:102720000813819504C0803F29F40E940813809308
:1027300086020895893F19F40E94471305C08A3F15
:1027400031F40E94471381958093880208958B3F4E
:1027500021F40E944713819504C08C3F29F40E9404
:1027600047138093890208959FE0980F983078F47A
:1027700021E030E0A90102C0440F551F9A95E2F70D
:10278000CA0190918502892B8093850208958D3F1F
:1027900021F48091830281600BC08E3F21F48091EF
:1027A0008302826005C08F3F29F480918302846098
:1027B0008093830208958D3E39F49091870297FFAC
:1027C00035C01092870259C08E3E29F4909187023D
:1027D0001916BCF32BC0909186028F3E29F497FF07
:1027E00025C01092860249C0803F19F41916CCF317
:1027F0001DC090918802893F29F41916BCF41092EB
:1028000088023BC08A3F19F497FF10C0F8CF8B3F76
:1028100039F49091890297FF09C0109289022DC066
:102820008C3F21F4909189021916BCF39FE0980F18
:10283000983080F421E030E0A90102C0440F551F18
:102840009A95E2F7CA018095909185028923809339
:10285000850213C08D3F21F4809183028E7F0BC0CF
:102860008E3F21F4809183028D7F05C08F3F29F434
:10287000809183028B7F80938302809186028111F5
:1028800006C080918702811102C01092820280915D
:102890008802811106C080918902811102C01092C4
:1028A000810208950E94951920918602211104C089
:1028B00020918702222321F09093800280937F024F
:1028C00020918802211104C020918902222321F045
:1028D00090937E0280937D0284E892E00C94FF172F
:1028E000EF92FF920F931F93CF93DF9300D000D00E
:1028F00000D0CDB7DEB786E0E4E8F2E0DE01119665
:1029000001900D928A95E1F7E0908602F09087029F
:10291000009188021091890210928602109287021B
:102920001092880210928902E11003C0FF2009F47E
:102930005DC080917F02909180020E94AD19AC0130
:1029400090918202992339F020910A0130E02417F6
:10295000350758F04BC020910B018AE0289F900169
:1029600011242417350718F041C09F3F19F09F5FCD
:1029700090938202EE2061F00E9408131E1414F05E
:102980009FEF01C091E0989F902D112490938602B3
:10299000FF2061F00E9408131F1414F09FEF01C084
:1029A00091E0989F902D1124909387023091860298
:1029B0003323E1F0209187022223C1F045EB340359
:1029C000C0011124992319F09093860203C081E07D
:1029D0008093860235EB2303C0011124992319F05B
:1029E0009093870203C081E080938702011103C0A6
:1029F000112309F45DC080917D0290917E020E94B6
:102A0000AD19AC0190918102992339F02091060112
:102A100030E02417350758F04BC0209107018AE0B9
:102A2000289F900111242417350718F041C09F3FBB
:102A300019F09F5F90938102002361F00E94471379
:102A4000101614F09FEF01C091E0989F902D112473
:102A500090938802112361F00E944713111614F01D
:102A60009FEF01C091E0989F902D112490938902CF
:102A7000309188023323E1F0209189022223C1F0B2
:102A800045EB3403C0011124992319F09093880277
:102A900003C081E08093880235EB2303C001112439
:102AA000992319F09093890203C081E080938902F1
:102AB0008091860281110BC080918702811107C02D
:102AC00080918802811103C08091890281110E9446
:102AD0005214EB82FC820D831E8386E0FE01319648
:102AE000A4E8B2E001900D928A95E1F726960FB620
:102AF000F894DEBF0FBECDBFDF91CF911F910F9134
:102B0000FF90EF900895E4E8F2E086E0DF011D9287
:102B10008A95E9F710928202109281021092830244
:102B20000895CF93DF93EC01FB018281882309F4A0
:102B30003CC1C430FDE5DF0760F4CB3F9CE5D9071D
:102B400088F49E0122503C452431310508F02EC105
:102B500009C0C236EDE5DE0729F0C63AFDE5DF071C
:102B600009F024C10E947E0D9093BC028093BB02A9
:102B7000C1318CE5D80709F4C6C008F042C0C9309D
:102B8000ECE5DE0709F49BC000F5C5308CE5D807FD
:102B900009F485C078F4C330ECE5DE0709F478C0A9
:102BA00008F07AC0C230DC4509F0F5C08091BB0264
:102BB0008160EFC0C7309CE5D90709F478C008F000
:102BC0007AC08091BB028061E4C0CD30FCE5DF07B4
:102BD00009F487C058F4CB309CE5D90709F479C0D3
:102BE00008F07BC08091BB0288606FC0CF30FCE5ED
:102BF000DF0709F480C008F082C08091BB02877FA4
:102C0000C8C0CE3F9CE5D90709F471C000F5C531B5
:102C1000FCE5DF0709F485C068F4C3319CE5D907FA
:102C200009F475C008F095C00E942F078091BB027F
:102C30008F77AFC0CC3FFCE5DF07A9F108F054C0A7
:102C4000CB3FDC4509F0A7C08091BC0240C0C23038
:102C5000EDE5DE0709F489C058F4C1158DE5D80704
:102C600009F45AC008F069C08091BC0282602FC08C
:102C7000C236EDE5DE0709F47CC0C63AFDE5DF07A4
:102C800009F481C0C330DD4509F085C080E06EC025
:102C90008091BB0282607DC08091BB0216C0809192
:102CA000BB02886076C08091BC0282604FC0809178
:102CB000BB0280626EC08091BB0280646AC00E94C9
:102CC0002F078091BB02806864C0846062C081600D
:102CD0003DC08091BB028E7F5CC08091BB028D7F26
:102CE00058C08091BB0216C08091BC0218C0809170
:102CF000BC028D7F2BC08091BB028F7E4AC0809129
:102D0000BB028F7D46C08091BB028F7B42C0809109
:102D1000BB02877F8B7F3DC08091BC028D7F8E7F01
:102D200015C08091BB0282FB222720F991E09227F7
:102D300090FB82F990FB83F92CC08091BC02982F04
:102D4000909591708E7F892B90FB81F98093BC02C6
:102D500022C00E942F078091BB0287FB222720F907
:102D600091E0922790FB87F914C081E00E94150E34
:102D700012C08091BB0284FB222720F991E09227A8
:102D800090FB84F906C08091BB02982F909590FB30
:102D900080F98093BB028091BB029091BC020E949B
:102DA0008F0D0E942F0780E001C081E0DF91CF915D
:102DB0000895CF93DF9386319C4541F5EB010E9446
:102DC000820C982F8A81209102013091030188237F
:102DD00079F09A7A81E009F480E080938A02911177
:102DE00002C069E201C065E3C9010E94CF180AC0B0
:102DF00080918A02811102C069E201C065E3C901C4
:102E00000E94DA180E94C40C80E001C081E0DF91CA
:102E1000CF9108950F931F93CF93DF93C42FD22F99
:102E2000FC0182818823C9F040938D020E9495198C
:102E300090938C0280938B0280E28C0F883008F094
:102E400057C0C77081E001C0880FCA95EAF7DF91CB
:102E5000CF911F910F910C948C0480918D02481397
:102E600030C080918B0290918C020E94AD19883CF9
:102E7000910538F510E21D0FCD17B9F080E28C0FE7
:102E8000883040F4C77081E001C0880FCA95EAF726
:102E90000E949304183028F581E09D2F977001C09F
:102EA000880F9A95EAF70E948C04802F0E94830471
:102EB0001830F0F4D77081E001C0880FDA95EAF796
:102EC0000AC080E28C0F883098F4C77081E001C09E
:102ED000880FCA95EAF7DF91CF911F910F910C945B
:102EE0009304802FDF91CF911F910F910C94830455
:102EF000DF91CF911F910F9108950F939C01CB010A
:102F0000243F4CE5340731F188F4293DFCE53F07C7
:102F1000D9F02A3D4CE5340779F1283D3C45A9F527
:102F200006E221EE41EE68ED7CE52BC0263FFCE594
:102F30003F07E1F0A8F0273F3C4539F507E225EED1
:102F400046EE67EF7CE51DC007E225EE45EE69ED34
:102F50007CE517C006E221EE40EE64EF7CE511C08F
:102F600007E225EE44EE65EF7CE50BC006E221EEBC
:102F700042EE66EF7CE505C008E221E045EE6AED31
:102F80007CE50E940A1780E008C0FC01828188234A
:102F900019F010928D0201C081E00F910895909375
:102FA00095018093940108959093930280939202E7
:102FB0000895E0919202F0919302309721F00190F0
:102FC000F081E02D099480E00895E0919202F09163
:102FD0009302309799F020911801222359F0209103
:102FE000BB0227FF07C0DC012C9111962C9311978F
:102FF00026E02C930280F381E02D09940895E0915E
:103000009202F0919302309739F022E0DC012C9388
:103010000480F581E02D099408952091900230916B
:1030200091022817390771F09093910280939002D2
:10303000E0919202F0919302309721F00680F7819F
:10304000E02D0994089520918E0230918F02281767
:10305000390771F090938F0280938E02E091920273
:10306000F0919302309721F00084F185E02D0994CE
:103070000895FC01329680911801882331F08091E7
:10308000BB0287FF02C09EE101C096E080E0915044
:1030900028F021912223D9F38F5FF9CF0895662379
:1030A00051F1209118012223E9F02091BB0227FF62
:1030B00019C0462F4695469546954E31E0F4677007
:1030C00021E030E002C0220F331F6A95E2F7FC01D5
:1030D000E40FF11D828190E02823392381E0232B26
:1030E00069F409C0FC01329608962191621729F013
:1030F000E817F907D1F780E0089581E008959C0171
:10310000FC0132969FEF80E04191461789F09F3F86
:1031100019F4411101C0982F8F5F8630A9F79F3FA6
:1031200039F0F901E90FF11D97FDFA9562830895D1
:1031300008959C012A5F3F4FFC014281461301C064
:103140001282019682179307B9F70895262F2695C4
:10315000269526952E3168F4FC01E20FF11D67706B
:1031600021E030E001C0220F6A95EAF78281282B26
:1031700022830895262F2695269526952E3170F4C4
:10318000FC01E20FF11D677021E030E001C0220F69
:103190006A95EAF720958281282322830895209159
:1031A0001801222329F02091BB0227FD0C94A618B8
:1031B0000C947F1820911801222329F02091BB0242
:1031C00027FD0C94BA180C94991820911801FC0151
:1031D0003296222331F08091BB0287FF02C08EE13C
:1031E00001C086E0DF011D928A95E9F708950895F0
:1031F0000C94F71883E0809394020C94F8188111D2
:1032000002C081E001C082E0809394020C94F8181F
:103210000C94FF1881E0809394020C94F8180C949D
:103220000A1908950C9411190C9412190C9411197F
:103230000C9411190C941119CF930E9418190E9423
:1032400067120E941619C0E08C2F0E947211672B22
:10325000682B692B29F4CF5FC530B1F780E001C03E
:1032600081E0CF91089508951F920F920FB60F92AB
:1032700011248F939F93AF93BF93809195028111F7
:1032800013C08091E5029091E602A091E702B0910F
:10329000E8024196A11DB11D8093E5029093E602DC
:1032A000A093E702B093E802BF91AF919F918F91F5
:1032B0000F900FBE0F901F9018958091ED028430F3
:1032C00031F10E94C4021092950220E488E190E05E
:1032D0000FB6F894A895809360000FBE209360000D
:1032E00083B7817F846083BF83B7816083BF789415
:1032F000889583B78E7F83BF0FB6F894A895809189
:103300006000886180936000109260000FBE089595
:103310000E942F070C94C80282E084BD93E095BD03
:103320009AEF97BD80936E0008952FB7F89480911F
:10333000E5029091E602A091E702B091E8022FBF6A
:1033400008952FB7F8946091E5027091E60280919C
:10335000E7029091E8022FBF08959C014FB7F894BF
:103360008091E5029091E602A091E702B091E80217
:103370004FBF821B930B089578941F920F920FB644
:103380000F9211248F939F93AF93BF938091E50287
:103390009091E602A091E702B091E8020196A11D8A
:1033A000B11D8093E5029093E602A093E702B093EB
:1033B000E802BF91AF919F918F910F900FBE0F9038
:1033C0001F901895F89481E08093E00080E280934C
:1033D000D800E9ECF0E010828FE19EE40197F1F76C
:1033E00000C000001DBA109268001CBC10BE1FBABD
:1033F00010927A0010926E0010926F00109270007E
:103400001092710010821092BC0011B814B817B855
:103410001AB81DB810BA12B815B818B81BB81EB82B
:1034200011BA0C9400FE08958091B9020895089590
:1034300022E02093E9002FEF3091E800215035FD84
:1034400006C035ED3A95F1F700002111F5CF209136
:10345000E80025FF0BC040E050E066E070E00E940D
:10346000551C8091E8008E778093E8000895CF93F3
:10347000DF9320911801222339F02091BB0227FF0E
:1034800003C060E222E002C068E021E02093E9008E
:103490002FEF3091E800215035FD06C035ED3A950B
:1034A000F1F700002111F5CF2091E80025FF1DC0A4
:1034B000EC0180911801811105C040E050E068E006
:1034C00070E003C070E040E050E0CE010E94551C67
:1034D0008091E8008E778093E80080E2FE01A9E900
:1034E000B2E001900D928A95E1F7DF91CF910895B6
:1034F0008093960270939802609397028091ED02F8
:10350000843001F582E08093E9008FEF9091E8002C
:10351000815095FD06C095ED9A95F1F70000811157
:10352000F5CF8091E80085FF0DC040E050E063E0FA
:1035300070E086E992E00E94551C8091E8008E7749
:103540008093E8000895BC0184E00C94781ABC01D3
:1035500083E00C94781A8091EC02811109C00E94DA
:10356000E21D0E94441E8091E20084608093E2008C
:1035700008951092EC0208950C940F196091E902DD
:1035800081E0611101C080E00C94FA189091ED0285
:1035900081E0943009F080E06091E9020C94FF181A
:1035A00042E061EC81E00E945B1D42E261EC82E05E
:1035B0000E945B1D9091ED0281E0943009F080E063
:1035C0006091E9020C9408198091EF02833009F4AC
:1035D0005FC030F4813071F0823009F498C00895F2
:1035E0008A3009F484C08B3009F46AC0893009F04C
:1035F000A6C020C08091EE02813A09F0A0C080915F
:10360000E800877F8093E8008091F2029091F302B6
:10361000892B21F460E289E992E003C060E080E058
:1036200090E070E00E94A01C8091E8008B7780936E
:10363000E80008958091EE02813209F080C0809107
:10364000F2029091F302029708F079C08091E800AD
:10365000877F8093E8008091E80082FD05C080911B
:10366000ED028111F8CF6BC08091F2009091F300D0
:10367000029731F48091F100813011F0863021F40D
:103680008091F1008093B9028091E8008B7753C05C
:103690008091EE02813A09F052C08091F20290913D
:1036A000F302892B09F04BC08091E800877F80935B
:1036B000E8008091E80080FFFCCF8091180136C0BF
:1036C0008091EE028132D9F58091F2029091F3025D
:1036D000892BA9F58091E800877F8093E8000E94FC
:1036E000901D8091F002809318010C942F07809117
:1036F000EE02813221F58091E800877F8093E80017
:103700000E94901D8091F1028093BA0208958091E9
:10371000EE02813AA1F48091E800877F8093E8006F
:103720008091E80080FFFCCF8091BA028093F10085
:103730008091E8008E778093E8000C94901D0895A6
:1037400084B7877F84BF0FB6F894A89580916000F6
:10375000886180936000109260000FBE90E080E866
:103760000FB6F89480936100909361000FBE0C94A3
:103770000A190E94E21D0E94441EE2EEF0E08081E0
:103780008460808378940C94DF208CE091E00C942A
:10379000D4178091ED028530A9F48091ED02853037
:1037A00079F40E945D198091EB028823B1F30E94A5
:1037B0001C19882391F30E943F1C0E942F07EDCF14
:1037C0000C948819089508950C94E61B292F33272B
:1037D00023303105C9F060F42130310581F0223009
:1037E000310509F044C08BE390E022E932E043C0A8
:1037F00021323105E1F02232310549F138C082E150
:1038000090E02DEC32E037C099278130910549F0E6
:1038100028F0029761F5E4E5F2E005C0EEE8F2E099
:1038200002C0EAE6F2E0849190E09F0124C06115B5
:10383000710541F061307105D1F489E090E02DEB24
:1038400032E019C089E090E024EA32E014C061154A
:10385000710541F06130710551F486EB90E02FED78
:1038600032E009C080E490E025E933E004C080E064
:1038700090E020E030E0FA0131832083089584E174
:1038800089BD86E189BD09B400FEFDCF8091D800D5
:103890008F7D8093D8008091E00082608093E0006B
:1038A0008091E00081FDFCCF0895CF92DF92EF92EE
:1038B000FF920F931F93CF93DF93EC018B017A015B
:1038C0000E94AF1D811133C0E114F10439F0F701FA
:1038D00080819181081B190BC80FD91FC12CD12CD5
:1038E0000115110519F18091E80085FD16C0809140
:1038F000E8008E778093E800E114F10449F0F701C5
:1039000080819181C80ED91ED182C08285E00FC00E
:103910000E94AF1D882321F30AC089918093F10092
:1039200001501109FFEFCF1ADF0ADACF80E0DF91F3
:10393000CF911F910F91FF90EF90DF90CF9008955E
:103940002091F4023091F5022617370748F06115EF
:10395000710539F42091E8002E772093E80001C02A
:10396000B901FC0120E06115710569F18091ED025A
:103970008823E1F18530E1F18091E80083FD3AC0D0
:103980008091E80082FD2CC08091E80080FFEBCFA1
:103990008091F2009091F3006115710551F088302B
:1039A000910538F421912093F1006150710901963D
:1039B000F3CF21E0089709F020E08091E8008E77AE
:1039C0008093E800D0CF2111D1CF0AC08091ED02C1
:1039D000882361F0853061F08091E80083FD0AC0A2
:1039E0008091E80082FFF2CF80E0089582E00895A0
:1039F00083E0089581E008952091F4023091F5026A
:103A00002617370748F06115710539F42091E80051
:103A10002E772093E80001C0B901FC0120E0611578
:103A2000710581F18091ED02882309F43EC0853053
:103A300009F43DC08091E80083FD3BC08091E8001F
:103A400082FD2DC08091E80080FFE9CF8091F200D7
:103A50009091F3006115710559F08830910540F49B
:103A600024912093F1003196615071090196F2CFB3
:103A700021E0089709F020E08091E8008E7780939C
:103A8000E800CDCF2111CECF0AC08091ED0288236E
:103A900061F0853061F08091E80083FD0AC080917B
:103AA000E80082FFF2CF80E0089582E0089583E08D
:103AB000089581E00895982F973068F59093E90074
:103AC000981739F07091EC002091ED005091F000C2
:103AD00003C0242F762F50E021FD02C09F5FECCF62
:103AE0003091EB003E7F3093EB003091ED003D7F55
:103AF0003093ED003091EB0031603093EB00709328
:103B0000EC002093ED005093F0002091EE0027FD93
:103B1000E5CF80E008958F708093E90081E00895FB
:103B20008091EE0287FF11C08091E80082FD05C000
:103B30008091ED028111F8CF11C08091E8008B7760
:103B40000BC08091ED02882349F08091E80080FF4E
:103B5000F8CF8091E8008E778093E8000895209157
:103B6000E4003091E50095E64091EC00842F8170EF
:103B700040FF23C08091E80080FD1DC08091ED02D0
:103B8000882399F0853099F08091EB0085FD11C074
:103B90004091E4005091E5002417350729F3915036
:103BA00011F09A01E1CF84E0089582E0089583E066
:103BB000089581E0089580E008954091E80042FF73
:103BC000DDCF08950E94531E0E945B1EE0EEF0E0E0
:103BD000808181608083E8EDF0E080818F77808351
:103BE00019BCA7EDB0E08C918E7F8C9380818F7E85
:103BF00080831092EC0208950F931F93CF93DF936D
:103C00000E94531E0E945B1EC8EDD0E088818F7712
:103C1000888388818068888388818F7D8883E7EDA9
:103C2000F0E080818068808319BC1092ED021092D0
:103C3000E9021092EB021092EA0200EE10E0F801A5
:103C400080818B7F808388818160888342E060E00F
:103C500080E00E945B1DE1EEF0E080818E7F80833A
:103C6000E2EEF0E0808181608083808188608083E3
:103C7000F80180818E7F8083888180618883DF91D5
:103C8000CF911F910F910895E8EDF0E080818F7E34
:103C90008083E7EDF0E080818160808381E0809324
:103CA000EC020C94FC1DE8EDF0E080818C7F8083B9
:103CB0001092E20008951092DA001092E100089547
:103CC0001F920F920FB60F9211240BB60F922F93E3
:103CD0003F934F935F936F937F938F939F93AF9394
:103CE000BF93EF93FF938091E10082FF0BC080911F
:103CF000E20082FF07C08091E1008B7F8093E100AA
:103D00000E94DE208091DA0080FF1FC08091D800E1
:103D100080FF1BC08091DA008E7F8093DA00809153
:103D2000D90080FF0DC084E189BD86E189BD09B459
:103D300000FEFDCF81E08093ED020E94AB1A05C02A
:103D400019BC1092ED020E94B91A8091E10080FF27
:103D500019C08091E20080FF15C08091E2008E7F43
:103D60008093E2008091E20080618093E200809184
:103D7000D80080628093D80019BC85E08093ED0262
:103D80000E94BE1A8091E10084FF30C08091E20061
:103D900084FF2CC084E189BD86E189BD09B400FEA1
:103DA000FDCF8091D8008F7D8093D8008091E10075
:103DB0008F7E8093E1008091E2008F7E8093E2000D
:103DC0008091E20081608093E2008091E902882383
:103DD00011F084E007C08091E30087FD02C081E01C
:103DE00001C083E08093ED020E94C61A8091E10039
:103DF00083FF29C08091E20083FF25C08091E1000C
:103E0000877F8093E10082E08093ED021092E902C7
:103E10008091E1008E7F8093E1008091E2008E7FAF
:103E20008093E2008091E20080618093E20042E0B2
:103E300060E080E00E945B1D8091F00088608093CC
:103E4000F0000E94BC1AFF91EF91BF91AF919F913A
:103E50008F917F916F915F914F913F912F910F9033
:103E60000BBE0F900FBE0F901F9018951F920F92D0
:103E70000FB60F9211240BB60F922F933F934F93CF
:103E80005F936F937F938F939F93AF93BF93CF93E2
:103E9000DF93EF93FF93C091E900CF708091EC0026
:103EA000D82FD17080FDD0E81092E9008091F00009
:103EB000877F8093F00078940E947E1F1092E90023
:103EC0008091F00088608093F000CD2BCF70C0937C
:103ED000E900FF91EF91DF91CF91BF91AF919F9159
:103EE0008F917F916F915F914F913F912F910F90A3
:103EF0000BBE0F900FBE0F901F9018951F93CF937E
:103F0000DF93CDB7DEB7AA970FB6F894DEBF0FBE2A
:103F1000CDBFEEEEF2E08091F100819322E0E63F2A
:103F2000F207C9F70E94E41A8091E80083FF2EC1CE
:103F30008091EE029091EF02492F50E04A305105F6
:103F400008F024C1FA01E85AFF4F0C940E21803882
:103F500021F0823809F01AC108C08091EA029091DC
:103F6000EB02992389F082600FC08091F2028F707A
:103F7000873008F00BC18093E9008091EB0085FB4E
:103F8000882780F91092E9009091E800977F90933C
:103F9000E8008093F1001092F100D1C0282F2D7F0E
:103FA00009F0F4C0882319F0823061F0EFC08091ED
:103FB000F002813009F0EAC0933009F080E080938C
:103FC000EB022EC08091F00281112AC08091F20292
:103FD0008F702FEF280F263008F0D8C08093E900AB
:103FE0002091EB0020FF1CC0933021F48091EB0066
:103FF000806214C09091EB0090619093EB0021E0FF
:1040000030E0A90102C0440F551F8A95E2F74093A2
:10401000EA001092EA008091EB0088608093EB0048
:104020001092E9008091E800877F8093E8000E9469
:10403000901DACC08111AAC01091F0021F77809131
:10404000E3008078812B8093E3008091E800877FF4
:104050008093E8000E94901D8091E80080FFFCCFD3
:104060008091E30080688093E300111102C082E038
:1040700001C083E08093ED0289C08058823008F04F
:1040800085C08091F0029091F1028C3D53E095073C
:1040900079F583E08A838AE289834FB7F894DE0159
:1040A000139620E03EE051E2E32FF0E050935700FA
:1040B000E49120FF03C0E295EF703F5FEF708E2F19
:1040C00090E0EA3010F0C79601C0C0968D939D93A2
:1040D0002F5F243149F74FBF8091E800877F80939D
:1040E000E8006AE270E0CE0101960E94A01C16C0B2
:1040F0006091F2027091F302AE014F5F5F4F0E9438
:10410000E41BBC01892B09F441C09091E800977F22
:104110009093E80089819A810E94FC1C8091E800BC
:104120008B778093E80032C0803881F58091E80079
:10413000877F8093E8008091E9028093F10080916D
:10414000E8008E7772CF811121C08091F0029091AA
:10415000F10299270297D4F48091E800877F809339
:10416000E8008091F0028093E9020E94901D809106
:10417000E902811106C08091E30087FD02C081E061
:1041800001C084E08093ED020E94D01A8091E80083
:1041900083FF0AC08091E800877F8093E8008091C8
:1041A000EB0080628093EB00AA960FB6F894DEBF16
:1041B0000FBECDBFDF91CF911F9108950895CF938A
:1041C0008091ED028823A1F0C091E900CF70909119
:1041D000EC00892F817090FD80E8C82B1092E900D7
:1041E0008091E80083FD0E947E1FCF70C093E9009C
:1041F000CF91089597FB072E16F4009407D077FD12
:1042000009D00E94172107FC05D03EF490958195B6
:104210009F4F0895709561957F4F0895EE0FFF1F92
:104220000024001C0BBE0790F691E02D0994AA1BF8
:10423000BB1B51E107C0AA1FBB1FA617B70710F091
:10424000A61BB70B881F991F5A95A9F780959095C3
:10425000BC01CD010895FB01DC0104C08D910190EA
:10426000801921F441505040C8F7881B990B0895DC
:10427000F999FECF92BD81BDF89A992780B508952E
:10428000A8E1B0E042E050E00C946C21262FF999AF
:10429000FECF92BD81BDF89A019700B4021639F0A5
:1042A0001FBA20BD0FB6F894FA9AF99A0FBE089576
:1042B0000396272F0E9447210E944621252F0E9406
:1042C0004721242F0C9447210196272F0E94472134
:1042D0000C944621DC01CB01FC01F999FECF06C00C
:1042E000F2BDE1BDF89A319600B40D9241505040B4
:0842F000B8F70895F894FFCF20
:1042F800C8003B02280850011E0A1401141A371A74
:10430800181AA71AA31A171A01E200E900EA00B559
:1043180000B600B700CD008301CC008A0192019459
:10432800012102230224022502260227022A02B3BF
:1043380000B4006F007000818283E200E900EA00A7
:10434800B500B600B700CD008301CC008A01920108
:1043580094012102230224022502260227022A02AE
:10436800B300B4006F00700081828390919293949F
:104378009597C067666564F0F1F2F3F4F5F6F763B4
:04438800626160C14D
:00000001FF
